:100000008316003085008600831258280130910045
:1000100001309200013093000130940001309500CE
:100020003D280830910004309200043093000230E3
:100030009400013095003D2840309100203092001E
:100040000830930004309400013095003D280030C2
:10005000910000309200603093001E309400013017
:1000600095003D2800309100003092000030930050
:10007000003094007F3095003D28851400008510E5
:1000800011088600502012088600502013088600B0
:1000900050201408860050201508860050200800C3
:1000A0009B0B502800308600051400000510080046
:1000B00050308C0006208C0B5A2840308C001120C8
:1000C0008C0B5F2830308C001C208C0B6428203077
:1000D0008C0027208C0B692810308C0032208C0B70
:0400E0006E28582806
:00000001FF
